 gpio

 Timestamp is 4da2a535 (Mon Apr 11 18:52:37 2011)

 Preferred load address is 10000000

 Start         Length     Name                   Class
 0001:00000000 00000004H .CRT$XCA                CODE
 0001:00000004 00000004H .CRT$XCZ                CODE
 0001:00000008 00000004H .CRT$XIA                CODE
 0001:0000000c 00000004H .CRT$XIZ                CODE
 0001:00000010 00000004H .CRT$XPA                CODE
 0001:00000014 00000004H .CRT$XPZ                CODE
 0001:00000018 00000004H .CRT$XTA                CODE
 0001:0000001c 00000004H .CRT$XTZ                CODE
 0001:00000020 00002b12H .rdata                  CODE
 0001:00002b34 00000021H .rdata$debug            CODE
 0001:00002b58 00003f18H .text                   CODE
 0001:00006a70 00000014H .xdata                  CODE
 0001:00006a84 00000028H .idata$2                CODE
 0001:00006aac 00000014H .idata$3                CODE
 0001:00006ac0 000000d4H .idata$4                CODE
 0001:00006b94 00000130H .idata$6                CODE
 0001:00006cd0 000000d8H .edata                  CODE
 0002:00000000 000000d4H .idata$5                DATA
 0002:000000d8 0000044cH .data                   DATA
 0002:00000528 00000fb4H .bss                    DATA
 0003:00000000 00000120H .pdata                  DATA

  Address         Publics by Value              Rva+Base       Lib:Object

 0000:00000000       ___safe_se_handler_count   00000000     <absolute>
 0000:00000000       ___safe_se_handler_table   00000000     <absolute>
 0001:00000000       __xc_a                     10001000     corelib0:crt0init.obj
 0001:00000004       __xc_z                     10001004     corelib0:crt0init.obj
 0001:00000008       __xi_a                     10001008     corelib0:crt0init.obj
 0001:0000000c       __xi_z                     1000100c     corelib0:crt0init.obj
 0001:00000010       __xp_a                     10001010     corelib0:crt0init.obj
 0001:00000014       __xp_z                     10001014     corelib0:crt0init.obj
 0001:00000018       __xt_a                     10001018     corelib0:crt0init.obj
 0001:0000001c       __xt_z                     1000101c     corelib0:crt0init.obj
 0001:00001040       ??_C@_1DO@CHLOKEDA@?$AAG?$AAP?$AAI?$AAO?$AA?5?$AAD?$AAr?$AAi?$AAv?$AAe?$AAr?$AA?3?$AA?5?$AA?9?$AAD?$AAl?$AAl?$AAM?$AAa?$AAi?$AAn?$AA?$CI?$AAT?$AAR?$AAU?$AAE?$AA?$CJ?$AA?9?$AA?$AN?$AA?6?$AA?$AA@ 10002040     Gpio.obj
 0001:00001080       ??_C@_1IA@BCJCPLH@?$AAG?$AAP?$AAI?$AAO?$AA?5?$AAD?$AAr?$AAi?$AAv?$AAe?$AAr?$AA?3?$AA?5?$AA?$CL?$AAD?$AAl?$AAl?$AAM?$AAa?$AAi?$AAn?$AA?$CI?$AAh?$AAI?$AAn?$AAs?$AAt?$AAa?$AAn?$AAc?$AAe?$AA?5@ 10002080     Gpio.obj
 0001:00001100       ??_C@_1DM@CFBFDENC@?$AAG?$AAP?$AAI?$AAO?$AA?5?$AAD?$AAr?$AAi?$AAv?$AAe?$AAr?$AA?3?$AA?5?$AA?9?$AAI?$AAn?$AAi?$AAt?$AA?$CI?$AA0?$AAx?$AA?$CF?$AA0?$AA8?$AAX?$AA?$CJ?$AA?9?$AA?$AN?$AA?6?$AA?$AA@ 10002100     Gpio.obj
 0001:00001140       ??_C@_1JK@CKNGKJEH@?$AAG?$AAP?$AAI?$AAO?$AA?5?$AAD?$AAr?$AAi?$AAv?$AAe?$AAr?$AA?3?$AA?5?$AA?5?$AAI?$AAn?$AAi?$AAt?$AA?$DO?$AA?5?$AAE?$AAR?$AAR?$AAO?$AAR?$AA?3?$AA?5?$AAC?$AAa?$AAn?$AA?8?$AAt@ 10002140     Gpio.obj
 0001:000011dc       ??_C@_1M@JJDCIKKN@?$AAP?$AAo?$AAr?$AAt?$AA4?$AA?$AA@ 100021dc     Gpio.obj
 0001:000011e8       ??_C@_1M@EOFLCBE@?$AAP?$AAo?$AAr?$AAt?$AA3?$AA?$AA@ 100021e8     Gpio.obj
 0001:000011f4       ??_C@_1M@LMFJNFHB@?$AAP?$AAo?$AAr?$AAt?$AA2?$AA?$AA@ 100021f4     Gpio.obj
 0001:00001200       ??_C@_1M@KOOMHKJP@?$AAP?$AAo?$AAr?$AAt?$AA1?$AA?$AA@ 10002200     Gpio.obj
 0001:00001210       ??_C@_1FO@HLOEDHBM@?$AAG?$AAP?$AAI?$AAO?$AA?5?$AAD?$AAr?$AAi?$AAv?$AAe?$AAr?$AA?3?$AA?5?$AA?$CL?$AAI?$AAn?$AAi?$AAt?$AA?$CI?$AAs?$AAz?$AAA?$AAc?$AAt?$AAi?$AAv?$AAe?$AAK?$AAe?$AAy?$AA?5?$AA?$DN@ 10002210     Gpio.obj
 0001:00001270       ??_C@_1DI@HHNHPFML@?$AAG?$AAP?$AAI?$AAO?$AA?5?$AAD?$AAr?$AAi?$AAv?$AAe?$AAr?$AA?3?$AA?5?$AA?9?$AAD?$AAe?$AAi?$AAn?$AAi?$AAt?$AA?$CI?$AA?$CF?$AAs?$AA?$CJ?$AA?9?$AA?$AN?$AA?6?$AA?$AA@ 10002270     Gpio.obj
 0001:000012a8       ??_C@_1M@HCOOECOK@?$AAF?$AAA?$AAL?$AAS?$AAE?$AA?$AA@ 100022a8     Gpio.obj
 0001:000012b4       ??_C@_19ELAAHEEL@?$AAT?$AAR?$AAU?$AAE?$AA?$AA@ 100022b4     Gpio.obj
 0001:000012c0       ??_C@_1FM@LKBKHFCD@?$AAG?$AAP?$AAI?$AAO?$AA?5?$AAD?$AAr?$AAi?$AAv?$AAe?$AAr?$AA?3?$AA?5?$AA?$CL?$AAD?$AAe?$AAi?$AAn?$AAi?$AAt?$AA?$CI?$AAp?$AAD?$AAr?$AAi?$AAv?$AAe?$AAr?$AAI?$AAn?$AAf?$AAo@ 100022c0     Gpio.obj
 0001:0000131c       ??_C@_1DM@EMMLGKOJ@?$AAG?$AAP?$AAI?$AAO?$AA?5?$AAD?$AAr?$AAi?$AAv?$AAe?$AAr?$AA?3?$AA?5?$AA?9?$AAO?$AAp?$AAe?$AAn?$AA?$CI?$AA0?$AAx?$AA?$CF?$AA0?$AA8?$AAX?$AA?$CJ?$AA?9?$AA?$AN?$AA?6?$AA?$AA@ 1000231c     Gpio.obj
 0001:00001358       ??_C@_1FI@OLFDNBDK@?$AAG?$AAP?$AAI?$AAO?$AA?5?$AAD?$AAr?$AAi?$AAv?$AAe?$AAr?$AA?3?$AA?5?$AA?5?$AAO?$AAp?$AAe?$AAn?$AA?$DO?$AA?5?$AAI?$AAN?$AAV?$AAA?$AAL?$AAI?$AAD?$AA_?$AAH?$AAA?$AAN?$AAD@ 10002358     Gpio.obj
 0001:000013b0       ??_C@_1JG@NGPDHDPJ@?$AAG?$AAP?$AAI?$AAO?$AA?5?$AAD?$AAr?$AAi?$AAv?$AAe?$AAr?$AA?3?$AA?5?$AA?5?$AAO?$AAp?$AAe?$AAn?$AA?$DO?$AA?5?$AAE?$AAR?$AAR?$AAO?$AAR?$AA?3?$AA?5?$AAC?$AAa?$AAn?$AA?8?$AAt@ 100023b0     Gpio.obj
 0001:00001448       ??_C@_1FI@MEPJJJCL@?$AAG?$AAP?$AAI?$AAO?$AA?5?$AAD?$AAr?$AAi?$AAv?$AAe?$AAr?$AA?3?$AA?5?$AA?$CL?$AAO?$AAp?$AAe?$AAn?$AA?$CI?$AAp?$AAD?$AAr?$AAi?$AAv?$AAe?$AAr?$AAI?$AAn?$AAf?$AAo?$AA?5?$AA?$DN@ 10002448     Gpio.obj
 0001:000014a0       ??_C@_1DM@DAHOCFLB@?$AAG?$AAP?$AAI?$AAO?$AA?5?$AAD?$AAr?$AAi?$AAv?$AAe?$AAr?$AA?3?$AA?5?$AA?9?$AAP?$AAr?$AAe?$AAC?$AAl?$AAo?$AAs?$AAe?$AA?$CI?$AA?$CF?$AAs?$AA?$CJ?$AA?9?$AA?$AN?$AA?6?$AA?$AA@ 100024a0     Gpio.obj
 0001:000014e0       ??_C@_1FM@BJONIFCP@?$AAG?$AAP?$AAI?$AAO?$AA?5?$AAD?$AAr?$AAi?$AAv?$AAe?$AAr?$AA?3?$AA?5?$AA?$CL?$AAP?$AAr?$AAe?$AAC?$AAl?$AAo?$AAs?$AAe?$AA?$CI?$AAp?$AAO?$AAp?$AAe?$AAn?$AAI?$AAn?$AAf?$AAo@ 100024e0     Gpio.obj
 0001:0000153c       ??_C@_1DG@FHBAADDN@?$AAG?$AAP?$AAI?$AAO?$AA?5?$AAD?$AAr?$AAi?$AAv?$AAe?$AAr?$AA?3?$AA?5?$AA?9?$AAC?$AAl?$AAo?$AAs?$AAe?$AA?$CI?$AA?$CF?$AAs?$AA?$CJ?$AA?9?$AA?$AN?$AA?6?$AA?$AA@ 1000253c     Gpio.obj
 0001:00001578       ??_C@_1FK@EPLHEAOO@?$AAG?$AAP?$AAI?$AAO?$AA?5?$AAD?$AAr?$AAi?$AAv?$AAe?$AAr?$AA?3?$AA?5?$AA?5?$AAC?$AAl?$AAo?$AAs?$AAe?$AA?$DO?$AA?5?$AAI?$AAN?$AAV?$AAA?$AAL?$AAI?$AAD?$AA_?$AAH?$AAA?$AAN@ 10002578     Gpio.obj
 0001:000015d8       ??_C@_1FG@OGAAIGCB@?$AAG?$AAP?$AAI?$AAO?$AA?5?$AAD?$AAr?$AAi?$AAv?$AAe?$AAr?$AA?3?$AA?5?$AA?$CL?$AAC?$AAl?$AAo?$AAs?$AAe?$AA?$CI?$AAp?$AAO?$AAp?$AAe?$AAn?$AAI?$AAn?$AAf?$AAo?$AA?5?$AA?$DN?$AA?5@ 100025d8     Gpio.obj
 0001:00001630       ??_C@_1DE@NBOAFCLK@?$AAG?$AAP?$AAI?$AAO?$AA?5?$AAD?$AAr?$AAi?$AAv?$AAe?$AAr?$AA?3?$AA?5?$AA?9?$AAR?$AAe?$AAa?$AAd?$AA?$CI?$AA?9?$AA1?$AA?$CJ?$AA?9?$AA?$AN?$AA?6?$AA?$AA@ 10002630     Gpio.obj
 0001:00001668       ??_C@_1FI@PCOIFIKF@?$AAG?$AAP?$AAI?$AAO?$AA?5?$AAD?$AAr?$AAi?$AAv?$AAe?$AAr?$AA?3?$AA?5?$AA?5?$AAR?$AAe?$AAa?$AAd?$AA?$DO?$AA?5?$AAI?$AAN?$AAV?$AAA?$AAL?$AAI?$AAD?$AA_?$AAH?$AAA?$AAN?$AAD@ 10002668     Gpio.obj
 0001:000016c0       ??_C@_1FE@GJFMNJGA@?$AAG?$AAP?$AAI?$AAO?$AA?5?$AAD?$AAr?$AAi?$AAv?$AAe?$AAr?$AA?3?$AA?5?$AA?5?$AAR?$AAe?$AAa?$AAd?$AA?$DO?$AA?5?$AAE?$AAR?$AAR?$AAO?$AAR?$AA_?$AAN?$AAO?$AAT?$AA_?$AAS?$AAU@ 100026c0     Gpio.obj
 0001:00001718       ??_C@_1FE@LPGNNIAP@?$AAG?$AAP?$AAI?$AAO?$AA?5?$AAD?$AAr?$AAi?$AAv?$AAe?$AAr?$AA?3?$AA?5?$AA?$CL?$AAR?$AAe?$AAa?$AAd?$AA?$CI?$AAp?$AAO?$AAp?$AAe?$AAn?$AAI?$AAn?$AAf?$AAo?$AA?5?$AA?$DN?$AA?5?$AA0@ 10002718     Gpio.obj
 0001:0000176c       ??_C@_1DG@LGDJBEAC@?$AAG?$AAP?$AAI?$AAO?$AA?5?$AAD?$AAr?$AAi?$AAv?$AAe?$AAr?$AA?3?$AA?5?$AA?9?$AAW?$AAr?$AAi?$AAt?$AAe?$AA?$CI?$AA?9?$AA1?$AA?$CJ?$AA?9?$AA?$AN?$AA?6?$AA?$AA@ 1000276c     Gpio.obj
 0001:000017a8       ??_C@_1FK@FNFCCHML@?$AAG?$AAP?$AAI?$AAO?$AA?5?$AAD?$AAr?$AAi?$AAv?$AAe?$AAr?$AA?3?$AA?5?$AA?5?$AAW?$AAr?$AAi?$AAt?$AAe?$AA?$DO?$AA?5?$AAI?$AAN?$AAV?$AAA?$AAL?$AAI?$AAD?$AA_?$AAH?$AAA?$AAN@ 100027a8     Gpio.obj
 0001:00001808       ??_C@_1FG@FHPIABFL@?$AAG?$AAP?$AAI?$AAO?$AA?5?$AAD?$AAr?$AAi?$AAv?$AAe?$AAr?$AA?3?$AA?5?$AA?5?$AAW?$AAr?$AAi?$AAt?$AAe?$AA?$DO?$AA?5?$AAE?$AAR?$AAR?$AAO?$AAR?$AA_?$AAN?$AAO?$AAT?$AA_?$AAS@ 10002808     Gpio.obj
 0001:00001860       ??_C@_1FG@BAHJIDH@?$AAG?$AAP?$AAI?$AAO?$AA?5?$AAD?$AAr?$AAi?$AAv?$AAe?$AAr?$AA?3?$AA?5?$AA?$CL?$AAW?$AAr?$AAi?$AAt?$AAe?$AA?$CI?$AAp?$AAO?$AAp?$AAe?$AAn?$AAI?$AAn?$AAf?$AAo?$AA?5?$AA?$DN?$AA?5@ 10002860     Gpio.obj
 0001:000018b8       ??_C@_1DE@OIFHHIKM@?$AAG?$AAP?$AAI?$AAO?$AA?5?$AAD?$AAr?$AAi?$AAv?$AAe?$AAr?$AA?3?$AA?5?$AA?9?$AAS?$AAe?$AAe?$AAk?$AA?$CI?$AA?9?$AA1?$AA?$CJ?$AA?9?$AA?$AN?$AA?6?$AA?$AA@ 100028b8     Gpio.obj
 0001:000018f0       ??_C@_1FI@EHDKIIME@?$AAG?$AAP?$AAI?$AAO?$AA?5?$AAD?$AAr?$AAi?$AAv?$AAe?$AAr?$AA?3?$AA?5?$AA?5?$AAS?$AAe?$AAe?$AAk?$AA?$DO?$AA?5?$AAI?$AAN?$AAV?$AAA?$AAL?$AAI?$AAD?$AA_?$AAH?$AAA?$AAN?$AAD@ 100028f0     Gpio.obj
 0001:00001948       ??_C@_1FE@NIFAKHJJ@?$AAG?$AAP?$AAI?$AAO?$AA?5?$AAD?$AAr?$AAi?$AAv?$AAe?$AAr?$AA?3?$AA?5?$AA?5?$AAS?$AAe?$AAe?$AAk?$AA?$DO?$AA?5?$AAE?$AAR?$AAR?$AAO?$AAR?$AA_?$AAN?$AAO?$AAT?$AA_?$AAS?$AAU@ 10002948     Gpio.obj
 0001:000019a0       ??_C@_1FE@OGBKGPG@?$AAG?$AAP?$AAI?$AAO?$AA?5?$AAD?$AAr?$AAi?$AAv?$AAe?$AAr?$AA?3?$AA?5?$AA?$CL?$AAS?$AAe?$AAe?$AAk?$AA?$CI?$AAp?$AAO?$AAp?$AAe?$AAn?$AAI?$AAn?$AAf?$AAo?$AA?5?$AA?$DN?$AA?5?$AA0@ 100029a0     Gpio.obj
 0001:000019f4       ??_C@_1DO@MKLPAJPA@?$AAG?$AAP?$AAI?$AAO?$AA?5?$AAD?$AAr?$AAi?$AAv?$AAe?$AAr?$AA?3?$AA?5?$AA?9?$AAI?$AAO?$AAC?$AAo?$AAn?$AAt?$AAr?$AAo?$AAl?$AA?$CI?$AA?$CF?$AAs?$AA?$CJ?$AA?9?$AA?$AN?$AA?6?$AA?$AA@ 100029f4     Gpio.obj
 0001:00001a38       ??_C@_1GA@LOKCFCLM@?$AAG?$AAP?$AAI?$AAO?$AA?5?$AAD?$AAr?$AAi?$AAv?$AAe?$AAr?$AA?3?$AA?5?$AA?5?$AAI?$AAO?$AAC?$AAo?$AAn?$AAt?$AAr?$AAo?$AAl?$AA?$DO?$AA?5?$AAE?$AAR?$AAR?$AAO?$AAR?$AA_?$AAI@ 10002a38     Gpio.obj
 0001:00001a98       ??_C@_1FO@IIBHCCHJ@?$AAG?$AAP?$AAI?$AAO?$AA?5?$AAD?$AAr?$AAi?$AAv?$AAe?$AAr?$AA?3?$AA?5?$AA?5?$AAI?$AAO?$AAC?$AAo?$AAn?$AAt?$AAr?$AAo?$AAl?$AA?$DO?$AA?5?$AAE?$AAR?$AAR?$AAO?$AAR?$AA_?$AAN@ 10002a98     Gpio.obj
 0001:00001af8       ??_C@_1IG@PKAMJOM@?$AAG?$AAP?$AAI?$AAO?$AA?5?$AAD?$AAr?$AAi?$AAv?$AAe?$AAr?$AA?3?$AA?5?$AA?5?$AAI?$AAO?$AAC?$AAo?$AAn?$AAt?$AAr?$AAo?$AAl?$AA?$DO?$AA?5?$AAI?$AAN?$AAF?$AAO?$AA?3?$AA?5?$AAG@ 10002af8     Gpio.obj
 0001:00001b80       ??_C@_1LE@PGFPDAGE@?$AAG?$AAP?$AAI?$AAO?$AA?5?$AAD?$AAr?$AAi?$AAv?$AAe?$AAr?$AA?3?$AA?5?$AA?5?$AAI?$AAO?$AAC?$AAo?$AAn?$AAt?$AAr?$AAo?$AAl?$AA?$DO?$AA?5?$AAE?$AAR?$AAR?$AAO?$AAR?$AA?3?$AA?5@ 10002b80     Gpio.obj
 0001:00001c38       ??_C@_1GA@ICGJFHAF@?$AAG?$AAP?$AAI?$AAO?$AA?5?$AAD?$AAr?$AAi?$AAv?$AAe?$AAr?$AA?3?$AA?5?$AA?5?$AAI?$AAO?$AAC?$AAo?$AAn?$AAt?$AAr?$AAo?$AAl?$AA?$DO?$AA?5?$AAI?$AAO?$AAC?$AAT?$AAL?$AA_?$AAG@ 10002c38     Gpio.obj
 0001:00001c98       ??_C@_1JC@IDJLBAPF@?$AAG?$AAP?$AAI?$AAO?$AA?5?$AAD?$AAr?$AAi?$AAv?$AAe?$AAr?$AA?3?$AA?5?$AA?5?$AAI?$AAO?$AAC?$AAo?$AAn?$AAt?$AAr?$AAo?$AAl?$AA?$DO?$AA?5?$AAI?$AAN?$AAF?$AAO?$AA?3?$AA?5?$AAU@ 10002c98     Gpio.obj
 0001:00001d2c       ??_C@_19CIJIHAKK@?$AAN?$AAU?$AAL?$AAL?$AA?$AA@ 10002d2c     Gpio.obj
 0001:00001d38       ??_C@_1IM@KNPMIOBF@?$AAG?$AAP?$AAI?$AAO?$AA?5?$AAD?$AAr?$AAi?$AAv?$AAe?$AAr?$AA?3?$AA?5?$AA?5?$AAI?$AAO?$AAC?$AAo?$AAn?$AAt?$AAr?$AAo?$AAl?$AA?$DO?$AA?5?$AAE?$AAR?$AAR?$AAO?$AAR?$AA?3?$AA?5@ 10002d38     Gpio.obj
 0001:00001dc8       ??_C@_1GO@HHBAHLHI@?$AAG?$AAP?$AAI?$AAO?$AA?5?$AAD?$AAr?$AAi?$AAv?$AAe?$AAr?$AA?3?$AA?5?$AA?5?$AAI?$AAO?$AAC?$AAo?$AAn?$AAt?$AAr?$AAo?$AAl?$AA?$DO?$AA?5?$AAI?$AAO?$AAC?$AAT?$AAL?$AA_?$AAG@ 10002dc8     Gpio.obj
 0001:00001e38       ??_C@_1IM@CILOOCKI@?$AAG?$AAP?$AAI?$AAO?$AA?5?$AAD?$AAr?$AAi?$AAv?$AAe?$AAr?$AA?3?$AA?5?$AA?5?$AAI?$AAO?$AAC?$AAo?$AAn?$AAt?$AAr?$AAo?$AAl?$AA?$DO?$AA?5?$AAI?$AAN?$AAF?$AAO?$AA?3?$AA?5?$AAE@ 10002e38     Gpio.obj
 0001:00001ec8       ??_C@_1LC@GOFDLKBE@?$AAG?$AAP?$AAI?$AAO?$AA?5?$AAD?$AAr?$AAi?$AAv?$AAe?$AAr?$AA?3?$AA?5?$AA?5?$AAI?$AAO?$AAC?$AAo?$AAn?$AAt?$AAr?$AAo?$AAl?$AA?$DO?$AA?5?$AAE?$AAR?$AAR?$AAO?$AAR?$AA?3?$AA?5@ 10002ec8     Gpio.obj
 0001:00001f80       ??_C@_1ME@MGKFICPB@?$AAG?$AAP?$AAI?$AAO?$AA?5?$AAD?$AAr?$AAi?$AAv?$AAe?$AAr?$AA?3?$AA?5?$AA?5?$AAI?$AAO?$AAC?$AAo?$AAn?$AAt?$AAr?$AAo?$AAl?$AA?$DO?$AA?5?$AAE?$AAR?$AAR?$AAO?$AAR?$AA?3?$AA?5@ 10002f80     Gpio.obj
 0001:00002048       ??_C@_1MC@GECGKJCP@?$AAG?$AAP?$AAI?$AAO?$AA?5?$AAD?$AAr?$AAi?$AAv?$AAe?$AAr?$AA?3?$AA?5?$AA?5?$AAI?$AAO?$AAC?$AAo?$AAn?$AAt?$AAr?$AAo?$AAl?$AA?$DO?$AA?5?$AAE?$AAR?$AAR?$AAO?$AAR?$AA?3?$AA?5@ 10003048     Gpio.obj
 0001:00002110       ??_C@_1GK@GBFLAIGP@?$AAG?$AAP?$AAI?$AAO?$AA?5?$AAD?$AAr?$AAi?$AAv?$AAe?$AAr?$AA?3?$AA?5?$AA?5?$AAI?$AAO?$AAC?$AAo?$AAn?$AAt?$AAr?$AAo?$AAl?$AA?$DO?$AA?5?$AAI?$AAO?$AAC?$AAT?$AAL?$AA_?$AAG@ 10003110     Gpio.obj
 0001:00002180       ??_C@_1GM@HOPHBACA@?$AAG?$AAP?$AAI?$AAO?$AA?5?$AAD?$AAr?$AAi?$AAv?$AAe?$AAr?$AA?3?$AA?5?$AA?5?$AAI?$AAO?$AAC?$AAo?$AAn?$AAt?$AAr?$AAo?$AAl?$AA?$DO?$AA?5?$AAI?$AAO?$AAC?$AAT?$AAL?$AA_?$AAG@ 10003180     Gpio.obj
 0001:000021f0       ??_C@_1GK@GPJAKJIA@?$AAG?$AAP?$AAI?$AAO?$AA?5?$AAD?$AAr?$AAi?$AAv?$AAe?$AAr?$AA?3?$AA?5?$AA?5?$AAI?$AAO?$AAC?$AAo?$AAn?$AAt?$AAr?$AAo?$AAl?$AA?$DO?$AA?5?$AAI?$AAO?$AAC?$AAT?$AAL?$AA_?$AAG@ 100031f0     Gpio.obj
 0001:00002260       ??_C@_1GK@BCGMDPDK@?$AAG?$AAP?$AAI?$AAO?$AA?5?$AAD?$AAr?$AAi?$AAv?$AAe?$AAr?$AA?3?$AA?5?$AA?5?$AAI?$AAO?$AAC?$AAo?$AAn?$AAt?$AAr?$AAo?$AAl?$AA?$DO?$AA?5?$AAI?$AAO?$AAC?$AAT?$AAL?$AA_?$AAG@ 10003260     Gpio.obj
 0001:000022d0       ??_C@_1GI@HBAFCAF@?$AAG?$AAP?$AAI?$AAO?$AA?5?$AAD?$AAr?$AAi?$AAv?$AAe?$AAr?$AA?3?$AA?5?$AA?5?$AAI?$AAO?$AAC?$AAo?$AAn?$AAt?$AAr?$AAo?$AAl?$AA?$DO?$AA?5?$AAI?$AAO?$AAC?$AAT?$AAL?$AA_?$AAG@ 100032d0     Gpio.obj
 0001:00002338       ??_C@_1GC@JEBGPJHG@?$AAG?$AAP?$AAI?$AAO?$AA?5?$AAD?$AAr?$AAi?$AAv?$AAe?$AAr?$AA?3?$AA?5?$AA?5?$AAI?$AAO?$AAC?$AAo?$AAn?$AAt?$AAr?$AAo?$AAl?$AA?$DO?$AA?5?$AAI?$AAO?$AAC?$AAT?$AAL?$AA_?$AAG@ 10003338     Gpio.obj
 0001:000023a0       ??_C@_1GA@DAOKMBAP@?$AAG?$AAP?$AAI?$AAO?$AA?5?$AAD?$AAr?$AAi?$AAv?$AAe?$AAr?$AA?3?$AA?5?$AA?5?$AAI?$AAO?$AAC?$AAo?$AAn?$AAt?$AAr?$AAo?$AAl?$AA?$DO?$AA?5?$AAI?$AAO?$AAC?$AAT?$AAL?$AA_?$AAG@ 100033a0     Gpio.obj
 0001:00002400       ??_C@_1GA@KPCGNBOJ@?$AAG?$AAP?$AAI?$AAO?$AA?5?$AAD?$AAr?$AAi?$AAv?$AAe?$AAr?$AA?3?$AA?5?$AA?5?$AAI?$AAO?$AAC?$AAo?$AAn?$AAt?$AAr?$AAo?$AAl?$AA?$DO?$AA?5?$AAI?$AAO?$AAC?$AAT?$AAL?$AA_?$AAG@ 10003400     Gpio.obj
 0001:00002460       ??_C@_1FO@FBNNDKBG@?$AAG?$AAP?$AAI?$AAO?$AA?5?$AAD?$AAr?$AAi?$AAv?$AAe?$AAr?$AA?3?$AA?5?$AA?5?$AAI?$AAO?$AAC?$AAo?$AAn?$AAt?$AAr?$AAo?$AAl?$AA?$DO?$AA?5?$AAI?$AAO?$AAC?$AAT?$AAL?$AA_?$AAG@ 10003460     Gpio.obj
 0001:000024c0       ??_C@_1GC@GMBPLKKK@?$AAG?$AAP?$AAI?$AAO?$AA?5?$AAD?$AAr?$AAi?$AAv?$AAe?$AAr?$AA?3?$AA?5?$AA?5?$AAI?$AAO?$AAC?$AAo?$AAn?$AAt?$AAr?$AAo?$AAl?$AA?$DO?$AA?5?$AAI?$AAO?$AAC?$AAT?$AAL?$AA_?$AAG@ 100034c0     Gpio.obj
 0001:00002528       ??_C@_1GC@OMNJHHAM@?$AAG?$AAP?$AAI?$AAO?$AA?5?$AAD?$AAr?$AAi?$AAv?$AAe?$AAr?$AA?3?$AA?5?$AA?5?$AAI?$AAO?$AAC?$AAo?$AAn?$AAt?$AAr?$AAo?$AAl?$AA?$DO?$AA?5?$AAI?$AAO?$AAC?$AAT?$AAL?$AA_?$AAG@ 10003528     Gpio.obj
 0001:00002590       ??_C@_1BAM@GPEDGBAN@?$AAG?$AAP?$AAI?$AAO?$AA?5?$AAD?$AAr?$AAi?$AAv?$AAe?$AAr?$AA?3?$AA?5?$AA?$CL?$AAI?$AAO?$AAC?$AAo?$AAn?$AAt?$AAr?$AAo?$AAl?$AA?$CI?$AAp?$AAO?$AAp?$AAe?$AAn?$AAI?$AAn?$AAf@ 10003590     Gpio.obj
 0001:000026a0       ??_C@_1EC@JKCGPNKL@?$AAG?$AAP?$AAI?$AAO?$AA?5?$AAD?$AAr?$AAi?$AAv?$AAe?$AAr?$AA?3?$AA?5?$AA?9?$AAS?$AAe?$AAt?$AAG?$AAp?$AAi?$AAo?$AAC?$AAo?$AAn?$AAf?$AAi?$AAg?$AA?$CI?$AA?$CJ?$AA?9?$AA?$AN?$AA?6@ 100036a0     Gpio.obj
 0001:000026e8       ??_C@_1IE@PBGHDDCG@?$AAG?$AAP?$AAI?$AAO?$AA?5?$AAD?$AAr?$AAi?$AAv?$AAe?$AAr?$AA?3?$AA?5?$AA?5?$AAS?$AAe?$AAt?$AAG?$AAp?$AAi?$AAo?$AAC?$AAo?$AAn?$AAf?$AAi?$AAg?$AA?$DO?$AA?5?$AAS?$AAe?$AAt@ 100036e8     Gpio.obj
 0001:00002770       ??_C@_1JE@OADDKOMH@?$AAG?$AAP?$AAI?$AAO?$AA?5?$AAD?$AAr?$AAi?$AAv?$AAe?$AAr?$AA?3?$AA?5?$AA?5?$AAS?$AAe?$AAt?$AAG?$AAp?$AAi?$AAo?$AAC?$AAo?$AAn?$AAf?$AAi?$AAg?$AA?$DO?$AA?5?$AAS?$AAe?$AAt@ 10003770     Gpio.obj
 0001:00002808       ??_C@_1IG@FKHLGAMN@?$AAG?$AAP?$AAI?$AAO?$AA?5?$AAD?$AAr?$AAi?$AAv?$AAe?$AAr?$AA?3?$AA?5?$AA?5?$AAS?$AAe?$AAt?$AAG?$AAp?$AAi?$AAo?$AAC?$AAo?$AAn?$AAf?$AAi?$AAg?$AA?$DO?$AA?5?$AAS?$AAe?$AAt@ 10003808     Gpio.obj
 0001:00002890       ??_C@_1IK@EBHFKBDM@?$AAG?$AAP?$AAI?$AAO?$AA?5?$AAD?$AAr?$AAi?$AAv?$AAe?$AAr?$AA?3?$AA?5?$AA?$CL?$AAS?$AAe?$AAt?$AAG?$AAp?$AAi?$AAo?$AAC?$AAo?$AAn?$AAf?$AAi?$AAg?$AA?$CI?$AAp?$AAG?$AAp?$AAi@ 10003890     Gpio.obj
 0001:00002920       ??_C@_1EC@HECEPDIN@?$AAG?$AAP?$AAI?$AAO?$AA?5?$AAD?$AAr?$AAi?$AAv?$AAe?$AAr?$AA?3?$AA?5?$AA?9?$AAG?$AAe?$AAt?$AAG?$AAp?$AAi?$AAo?$AAC?$AAo?$AAn?$AAf?$AAi?$AAg?$AA?$CI?$AA?$CJ?$AA?9?$AA?$AN?$AA?6@ 10003920     Gpio.obj
 0001:00002968       ??_C@_1GO@MDKMBDFB@?$AAG?$AAP?$AAI?$AAO?$AA?5?$AAD?$AAr?$AAi?$AAv?$AAe?$AAr?$AA?3?$AA?5?$AA?5?$AAG?$AAe?$AAt?$AAG?$AAp?$AAi?$AAo?$AAC?$AAo?$AAn?$AAf?$AAi?$AAg?$AA?$DO?$AA?5?$AAG?$AAP?$AAI@ 10003968     Gpio.obj
 0001:000029d8       ??_C@_1HO@KMCFPBAO@?$AAG?$AAP?$AAI?$AAO?$AA?5?$AAD?$AAr?$AAi?$AAv?$AAe?$AAr?$AA?3?$AA?5?$AA?5?$AAG?$AAe?$AAt?$AAG?$AAp?$AAi?$AAo?$AAC?$AAo?$AAn?$AAf?$AAi?$AAg?$AA?$DO?$AA?5?$AAG?$AAP?$AAI@ 100039d8     Gpio.obj
 0001:00002a58       ??_C@_1HA@IOJDNPLF@?$AAG?$AAP?$AAI?$AAO?$AA?5?$AAD?$AAr?$AAi?$AAv?$AAe?$AAr?$AA?3?$AA?5?$AA?5?$AAG?$AAe?$AAt?$AAG?$AAp?$AAi?$AAo?$AAC?$AAo?$AAn?$AAf?$AAi?$AAg?$AA?$DO?$AA?5?$AAG?$AAP?$AAI@ 10003a58     Gpio.obj
 0001:00002ac8       ??_C@_1GK@PDPHGFBA@?$AAG?$AAP?$AAI?$AAO?$AA?5?$AAD?$AAr?$AAi?$AAv?$AAe?$AAr?$AA?3?$AA?5?$AA?$CL?$AAG?$AAe?$AAt?$AAG?$AAp?$AAi?$AAo?$AAC?$AAo?$AAn?$AAf?$AAi?$AAg?$AA?$CI?$AAp?$AAG?$AAp?$AAi@ 10003ac8     Gpio.obj
 0001:00002b58       ?to_T@@YAPBGPBD@Z          10003b58 f   DebugZones.obj
 0001:00002bf4       DllMain                    10003bf4 f   Gpio.obj
 0001:00002ca8       ?GpioIntrThread@@YAKPAX@Z  10003ca8 f   Gpio.obj
 0001:00002d64       ?CleanInterruptHandler@@YAXPAUINTR_INFO@@@Z 10003d64 f   Gpio.obj
 0001:00002eac       ?SetupInterruptHandler@@YAHPAUINTR_INFO@@@Z 10003eac f   Gpio.obj
 0001:0000312c       ?Init@@YAPAUDRIVER_INFO@@PAX@Z 1000412c f   Gpio.obj
 0001:000033d4       ?Deinit@@YAHPAUDRIVER_INFO@@@Z 100043d4 f   Gpio.obj
 0001:000034ec       ?Open@@YAPAUOPEN_INFO@@PAUDRIVER_INFO@@KK@Z 100044ec f   Gpio.obj
 0001:000036f0       ?PreClose@@YAHPAUOPEN_INFO@@@Z 100046f0 f   Gpio.obj
 0001:00003834       ?Close@@YAHPAUOPEN_INFO@@@Z 10004834 f   Gpio.obj
 0001:00003970       ?Read@@YAKPAUOPEN_INFO@@PAEK@Z 10004970 f   Gpio.obj
 0001:00003ae0       ?Write@@YAKPAUOPEN_INFO@@PAEK@Z 10004ae0 f   Gpio.obj
 0001:00003c50       ?Seek@@YAKPAUOPEN_INFO@@JK@Z 10004c50 f   Gpio.obj
 0001:00003dc0       ?IOControl@@YAHPAUOPEN_INFO@@KPAEK1KPAK@Z 10004dc0 f   Gpio.obj
 0001:00005090       ?PowerUp@@YAHPAUDRIVER_INFO@@@Z 10006090 f   Gpio.obj
 0001:000050b4       ?PowerDown@@YAHPAUDRIVER_INFO@@@Z 100060b4 f   Gpio.obj
 0001:00006064       SetEvent                   10007064 f i Gpio.obj
 0001:00006098       GetCurrentThread           10007098 f i Gpio.obj
 0001:000060b0       RegisterDbgZones           100070b0 f   coredll:COREDLL.dll
 0001:000060c0       DisableThreadLibraryCalls  100070c0 f   coredll:COREDLL.dll
 0001:000060d0       NKDbgPrintfW               100070d0 f   coredll:COREDLL.dll
 0001:000060e0       InterruptDone              100070e0 f   coredll:COREDLL.dll
 0001:000060f0       WaitForSingleObject        100070f0 f   coredll:COREDLL.dll
 0001:00006100       CeSetThreadPriority        10007100 f   coredll:COREDLL.dll
 0001:00006110       EventModify                10007110 f   coredll:COREDLL.dll
 0001:00006120       CloseHandle                10007120 f   coredll:COREDLL.dll
 0001:00006130       TerminateThread            10007130 f   coredll:COREDLL.dll
 0001:00006140       InterruptDisable           10007140 f   coredll:COREDLL.dll
 0001:00006150       KernelIoControl            10007150 f   coredll:COREDLL.dll
 0001:00006160       CreateThread               10007160 f   coredll:COREDLL.dll
 0001:00006170       InterruptInitialize        10007170 f   coredll:COREDLL.dll
 0001:00006180       CreateEventW               10007180 f   coredll:COREDLL.dll
 0001:00006190       GetLastError               10007190 f   coredll:COREDLL.dll
 0001:000061a0       RegCloseKey                100071a0 f   coredll:COREDLL.dll
 0001:000061b0       RegQueryValueExW           100071b0 f   coredll:COREDLL.dll
 0001:000061c0       OpenDeviceKey              100071c0 f   coredll:COREDLL.dll
 0001:000061d0       InitializeCriticalSection  100071d0 f   coredll:COREDLL.dll
 0001:000061e0       DeleteCriticalSection      100071e0 f   coredll:COREDLL.dll
 0001:000061f0       SetLastError               100071f0 f   coredll:COREDLL.dll
 0001:00006200       LeaveCriticalSection       10007200 f   coredll:COREDLL.dll
 0001:00006210       EnterCriticalSection       10007210 f   coredll:COREDLL.dll
 0001:00006220       DDKGpioClearIntrPin        10007220 f   cspddk:CSPDDK.dll
 0001:00006230       DDKGpioReadIntr            10007230 f   cspddk:CSPDDK.dll
 0001:00006240       DDKGpioReadIntrPin         10007240 f   cspddk:CSPDDK.dll
 0001:00006250       DDKGpioWriteData           10007250 f   cspddk:CSPDDK.dll
 0001:00006260       DDKGpioReadData            10007260 f   cspddk:CSPDDK.dll
 0001:00006270       DDKGpioWriteDataPin        10007270 f   cspddk:CSPDDK.dll
 0001:00006280       DDKGpioReadDataPin         10007280 f   cspddk:CSPDDK.dll
 0001:00006290       DDKGpioSetConfig           10007290 f   cspddk:CSPDDK.dll
 0001:000062a0       DDKIomuxSetPadConfigPort   100072a0 f   cspddk:CSPDDK.dll
 0001:000062b0       DDKIomuxSetPinMux          100072b0 f   cspddk:CSPDDK.dll
 0001:000062c0       DDKGpioGetConfig           100072c0 f   cspddk:CSPDDK.dll
 0001:000062d0       DDKIomuxGetPadConfigPort   100072d0 f   cspddk:CSPDDK.dll
 0001:000062e0       DDKIomuxGetPinMux          100072e0 f   cspddk:CSPDDK.dll
 0001:000062f0       _DllMainCRTStartup         100072f0 f   corelib0:pegdmain.obj
 0001:00006488       __security_init_cookie     10007488 f   corelib0:seccinit.obj
 0001:00006520       exit                       10007520 f   corelib0:cexit.obj
 0001:00006644       _exit                      10007644 f   corelib0:cexit.obj
 0001:00006664       _cexit                     10007664 f   corelib0:cexit.obj
 0001:0000667c       _c_exit                    1000767c f   corelib0:cexit.obj
 0001:00006694       _initterm                  10007694 f   corelib0:crt0dat.obj
 0001:000066e0       _cinit                     100076e0 f   corelib0:crt0dat.obj
 0001:00006710       __crt_ExitProcess          10007710 f   corelib0:exitproc_proxy.obj
 0001:0000673c       GetCurrentProcess          1000773c f i corelib0:exitproc_proxy.obj
 0001:00006754       _onexit                    10007754 f   corelib0:onexit.obj
 0001:00006930       atexit                     10007930 f   corelib0:onexit.obj
 0001:00006980       mbstowcs                   10007980 f   corelib1:COREDLL.dll
 0001:00006990       _wcsdup                    10007990 f   corelib1:COREDLL.dll
 0001:000069a0       memset                     100079a0 f   corelib1:COREDLL.dll
 0001:000069b0       ??2@YAPAXI@Z               100079b0 f   corelib1:COREDLL.dll
 0001:000069c0       ??3@YAXPAX@Z               100079c0 f   corelib1:COREDLL.dll
 0001:000069d0       free                       100079d0 f   corelib1:COREDLL.dll
 0001:000069e0       wcscpy                     100079e0 f   corelib1:COREDLL.dll
 0001:000069f0       memcpy                     100079f0 f   corelib1:COREDLL.dll
 0001:00006a00       _XcptFilter                10007a00 f   corelib1:COREDLL.dll
 0001:00006a10       __C_specific_handler       10007a10 f   corelib1:COREDLL.dll
 0001:00006a20       __security_gen_cookie2     10007a20 f   corelib1:COREDLL.dll
 0001:00006a30       realloc                    10007a30 f   corelib1:COREDLL.dll
 0001:00006a40       malloc                     10007a40 f   corelib1:COREDLL.dll
 0001:00006a50       _msize                     10007a50 f   corelib1:COREDLL.dll
 0001:00006a60       TerminateProcess           10007a60 f   coredll:COREDLL.dll
 0001:00006a84       __IMPORT_DESCRIPTOR_COREDLL 10007a84     coredll:COREDLL.dll
 0001:00006a98       __IMPORT_DESCRIPTOR_CSPDDK 10007a98     cspddk:CSPDDK.dll
 0001:00006aac       __NULL_IMPORT_DESCRIPTOR   10007aac     coredll:COREDLL.dll
 0002:00000000       __imp_RegisterDbgZones     10008000     coredll:COREDLL.dll
 0002:00000004       __imp_DisableThreadLibraryCalls 10008004     coredll:COREDLL.dll
 0002:00000008       __imp_NKDbgPrintfW         10008008     coredll:COREDLL.dll
 0002:0000000c       __imp_InterruptDone        1000800c     coredll:COREDLL.dll
 0002:00000010       __imp_WaitForSingleObject  10008010     coredll:COREDLL.dll
 0002:00000014       __imp_CeSetThreadPriority  10008014     coredll:COREDLL.dll
 0002:00000018       __imp_EventModify          10008018     coredll:COREDLL.dll
 0002:0000001c       __imp_CloseHandle          1000801c     coredll:COREDLL.dll
 0002:00000020       __imp_TerminateThread      10008020     coredll:COREDLL.dll
 0002:00000024       __imp_InterruptDisable     10008024     coredll:COREDLL.dll
 0002:00000028       __imp_KernelIoControl      10008028     coredll:COREDLL.dll
 0002:0000002c       __imp_CreateThread         1000802c     coredll:COREDLL.dll
 0002:00000030       __imp_InterruptInitialize  10008030     coredll:COREDLL.dll
 0002:00000034       __imp_CreateEventW         10008034     coredll:COREDLL.dll
 0002:00000038       __imp_GetLastError         10008038     coredll:COREDLL.dll
 0002:0000003c       __imp_RegCloseKey          1000803c     coredll:COREDLL.dll
 0002:00000040       __imp_RegQueryValueExW     10008040     coredll:COREDLL.dll
 0002:00000044       __imp_OpenDeviceKey        10008044     coredll:COREDLL.dll
 0002:00000048       __imp_InitializeCriticalSection 10008048     coredll:COREDLL.dll
 0002:0000004c       __imp_DeleteCriticalSection 1000804c     coredll:COREDLL.dll
 0002:00000050       __imp_SetLastError         10008050     coredll:COREDLL.dll
 0002:00000054       __imp_LeaveCriticalSection 10008054     coredll:COREDLL.dll
 0002:00000058       __imp_EnterCriticalSection 10008058     coredll:COREDLL.dll
 0002:0000005c       __imp__msize               1000805c     corelib1:COREDLL.dll
 0002:00000060       __imp_malloc               10008060     corelib1:COREDLL.dll
 0002:00000064       __imp_TerminateProcess     10008064     coredll:COREDLL.dll
 0002:00000068       __imp_realloc              10008068     corelib1:COREDLL.dll
 0002:0000006c       __imp___security_gen_cookie2 1000806c     corelib1:COREDLL.dll
 0002:00000070       __imp___C_specific_handler 10008070     corelib1:COREDLL.dll
 0002:00000074       __imp__XcptFilter          10008074     corelib1:COREDLL.dll
 0002:00000078       __imp_memcpy               10008078     corelib1:COREDLL.dll
 0002:0000007c       __imp_wcscpy               1000807c     corelib1:COREDLL.dll
 0002:00000080       __imp_free                 10008080     corelib1:COREDLL.dll
 0002:00000084       __imp_??3@YAXPAX@Z         10008084     corelib1:COREDLL.dll
 0002:00000088       __imp_??2@YAPAXI@Z         10008088     corelib1:COREDLL.dll
 0002:0000008c       __imp_memset               1000808c     corelib1:COREDLL.dll
 0002:00000090       __imp__wcsdup              10008090     corelib1:COREDLL.dll
 0002:00000094       __imp_mbstowcs             10008094     corelib1:COREDLL.dll
 0002:00000098       \177COREDLL_NULL_THUNK_DATA 10008098     coredll:COREDLL.dll
 0002:0000009c       __imp_DDKIomuxGetPinMux    1000809c     cspddk:CSPDDK.dll
 0002:000000a0       __imp_DDKIomuxGetPadConfigPort 100080a0     cspddk:CSPDDK.dll
 0002:000000a4       __imp_DDKGpioGetConfig     100080a4     cspddk:CSPDDK.dll
 0002:000000a8       __imp_DDKIomuxSetPinMux    100080a8     cspddk:CSPDDK.dll
 0002:000000ac       __imp_DDKIomuxSetPadConfigPort 100080ac     cspddk:CSPDDK.dll
 0002:000000b0       __imp_DDKGpioSetConfig     100080b0     cspddk:CSPDDK.dll
 0002:000000b4       __imp_DDKGpioReadDataPin   100080b4     cspddk:CSPDDK.dll
 0002:000000b8       __imp_DDKGpioWriteDataPin  100080b8     cspddk:CSPDDK.dll
 0002:000000bc       __imp_DDKGpioReadData      100080bc     cspddk:CSPDDK.dll
 0002:000000c0       __imp_DDKGpioWriteData     100080c0     cspddk:CSPDDK.dll
 0002:000000c4       __imp_DDKGpioReadIntr      100080c4     cspddk:CSPDDK.dll
 0002:000000c8       __imp_DDKGpioClearIntrPin  100080c8     cspddk:CSPDDK.dll
 0002:000000cc       __imp_DDKGpioReadIntrPin   100080cc     cspddk:CSPDDK.dll
 0002:000000d0       \177CSPDDK_NULL_THUNK_DATA 100080d0     cspddk:CSPDDK.dll
 0002:000000d8       dpCurSettings              100080d8     DebugZones.obj
 0002:0000051c       __security_cookie          1000851c     corelib0:seccinit.obj
 0002:00000520       __security_cookie_complement 10008520     corelib0:seccinit.obj
 0002:000014cc       _exitflag                  100094cc     corelib0:cexit.obj
 0002:000014d0       __onexitend                100094d0     <common>
 0002:000014d4       __onexitbegin              100094d4     <common>
 0002:000014d8       _pRawDllMain               100094d8     <common>

 entry point at        0001:000062f0

 Static symbols

 0001:000050d8       ?SetGpioConfig@@YAXPAUGPIO_CONFIG@@@Z 100060d8 f   Gpio.obj
 0001:000050f4       ?SetGpioConfig@@YAXPAUGPIO_CONFIG@@H@Z 100060f4 f   Gpio.obj
 0001:000057c0       ?GetGpioConfig@@YAXPAUGPIO_CONFIG@@@Z 100067c0 f   Gpio.obj
 0001:00006340       _DllMainCRTStartupHelper   10007340 f   corelib0:pegdmain.obj
 0001:00006540       doexit                     10007540 f   corelib0:cexit.obj
